:0200000480007A
:100000006F000005732F2034930F80006308FF03F7
:10001000930F90006304FF03930FB0006300FF038E
:10002000130F000063040F0067000F00732F2034CC
:1000300063540F006F00400093E19153171F0000BD
:1000400023223FFC171F000023200FFC6FF01FFF2F
:100050009300000013010000930100001302000050
:100060009302000013030000930300001304000038
:100070009304000013050000930500001306000020
:100080009306000013070000930700001308000008
:10009000930800001309000093090000130A0000F0
:1000A000930A0000130B0000930B0000130C0000D8
:1000B000930C0000130D0000930D0000130E0000C0
:1000C000930E0000130F0000930F0000732540F102
:1000D0006310050097020000938202017390523072
:1000E000735044749702000093820201739052305F
:1000F00073500018970200009382420273905230AE
:100100009B021000939252039382F2FF7390023B82
:100110009302F0017390023A73504030970200004E
:1001200093824201739052307350203073503030BC
:100130009301000097020000938202ED7390523009
:10014000130510001315F501635C05000F00F00F97
:10015000930110009308D005130500007300000000
:1001600093020000638A020073905210B7B200003D
:100170009B829210739022307350003097020000DF
:100180009382420173901234732540F17300203042
:1001900093012000B70001009B8010F093900001B4
:1001A000938000F037110F0F1B01F1F033E72000AF
:1001B000B71300009B8313FF939343019383F3F0E2
:1001C0006316775A93013000B710F00F9B8000FF41
:1001D00037110F001B01F1F01311C1001301010FC2
:1001E00033E72000B70301009B8313FF93930301C0
:1001F000938303FF631C775693014000B700FF0011
:100200009B80F00F37110F0F1B01F1F033E7200037
:10021000B713FF0F9B83F3FF631A775493015000CA
:10022000B7000F009B80F00F9390C0009380F00008
:1002300037110F001B01F1F01311C1001301010F61
:1002400033E72000B7130F009B83F3FF9393C300A2
:100250009383F30F631C775093016000B700010094
:100260009B8010F093900001938000F037110F0FE6
:100270001B01F1F0B3E02000B71300009B8313FFD4
:10028000939343019383F3F06392704E9301700054
:10029000B70001009B8010F093900001938000F064
:1002A00037110F0F1B01F1F033E12000B7130000ED
:1002B0009B8313FF939343019383F3F06318714A75
:1002C00093018000B70001009B8010F09390000123
:1002D000938000F0B3E01000B70301009B8313F09C
:1002E00093930301938303F063927048930190000A
:1002F00013020000B70001009B8010F093900001F2
:10030000938000F037110F0F1B01F1F033E720004D
:10031000130307001302120093022000E31C52FC97
:10032000B71300009B8313FF939343019383F3F070
:10033000631E73429301A00013020000B710F00F78
:100340009B8000FF37110F001B01F1F01311C1005A
:100350001301010F33E7200013000000130307000F
:100360001302120093022000E31A52FCB7030100AB
:100370009B8313FF93930301938303FF6318733EDF
:100380009301B00013020000B700FF009B80F00F44
:1003900037110F0F1B01F1F033E7200013000000AD
:1003A0001300000013030700130212009302200041
:1003B000E31C52FCB713FF0F9B83F3FF6318733AE0
:1003C0009301C00013020000B70001009B8010F0F1
:1003D00093900001938000F037110F0F1B01F1F093
:1003E00033E720001302120093022000E31E52FCA8
:1003F000B71300009B8313FF939343019383F3F0A0
:10040000631677369301D00013020000B710F00F87
:100410009B8000FF37110F001B01F1F01311C10089
:100420001301010F1300000033E720001302120034
:1004300093022000E31C52FCB70301009B8313FFCF
:1004400093930301938303FF631277329301E000D8
:1004500013020000B700FF009B80F00F37110F0F51
:100460001B01F1F0130000001300000033E720002F
:100470001302120093022000E31E52FCB713FF0F79
:100480009B83F3FF6314772E9301F00013020000A7
:10049000B70001009B8010F093900001938000F062
:1004A0001300000037110F0F1B01F1F033E720009C
:1004B0001302120093022000E31C52FCB713000049
:1004C0009B8313FF939343019383F3F06310772A85
:1004D0009301000113020000B710F00F9B8000FF92
:1004E0001300000037110F001B01F1F01311C100C0
:1004F0001301010F1300000033E720001302120064
:1005000093022000E31A52FCB70301009B8313FF00
:1005100093930301938303FF631A772493011001DC
:1005200013020000B700FF009B80F00F13000000D3
:100530001300000037110F0F1B01F1F033E720000B
:100540001302120093022000E31E52FCB713FF0FA8
:100550009B83F3FF631C77209301200113020000AB
:1005600037110F0F1B01F1F0B70001009B8010F055
:1005700093900001938000F033E7200013021200F3
:1005800093022000E31E52FCB71300009B8313FF6D
:10059000939343019383F3F0631A771C9301300123
:1005A0001302000037110F001B01F1F01311C100FD
:1005B0001301010FB710F00F9B8000FF1300000024
:1005C00033E720001302120093022000E31C52FCC8
:1005D000B70301009B8313FF93930301938303FFEE
:1005E00063167718930140011302000037110F0FB3
:1005F0001B01F1F0B700FF009B80F00F130000001B
:100600001300000033E720001302120093022000C1
:10061000E31E52FCB713FF0F9B83F3FF631877149D
:10062000930150011302000037110F0F1B01F1F06D
:1006300013000000B70001009B8010F093900001B0
:10064000938000F033E72000130212009302200091
:10065000E31C52FCB71300009B8313FF93934301E9
:100660009383F3F063147710930160011302000089
:1006700037110F001B01F1F01311C1001301010F1D
:1006800013000000B710F00F9B8000FF1300000064
:1006900033E720001302120093022000E31A52FCF9
:1006A000B70301009B8313FF93930301938303FF1D
:1006B000631E770A930170011302000037110F0FB8
:1006C0001B01F1F01300000013000000B700FF0051
:1006D0009B80F00F33E720001302120093022000EA
:1006E000E31E52FCB713FF0F9B83F3FF63107708E1
:1006F00093018001B70001009B8010F093900001EE
:10070000938000F033611000B70301009B8313F066
:1007100093930301938303F0631A7104930190018F
:10072000B700FF009B80F00F33E10000B703FF002C
:100730009B83F30F631C71029301A001B36000005F
:1007400093030000639470029301B001B71011117C
:100750009B801011372122221B01212233E020002F
:100760009303000063147000631030020F00F00F59
:10077000638001009391110093E111009308D0056B
:1007800013850100730000000F00F00F93011000AB
:100790009308D0051305000073000000731000C01B
:1007A0000000000000000000000000000000000049
:0C07B0000000000000000000000000003D
:1010000000000000000000000000000000000000E0
:1010100000000000000000000000000000000000D0
:1010200000000000000000000000000000000000C0
:1010300000000000000000000000000000000000B0
:081040000000000000000000A8
:040000058000000077
:00000001FF
